:020000020000FC
:100000000C946123189518951895189518951895BE
:100010001895189518951895189518951895189578
:100020001895189518951895189518951895189568
:100030001895189518951895189518951895189558
:100040001895189518951895189518951895189548
:100050000C94D50818951895189518951895189515
:100060001895189518951895189518951895189528
:100070001895189518951895189518951895189518
:100080001895189518951895189518951895189508
:1000900018951895189518951895189518951895F8
:1000A00018951895189518951895189518951895E8
:1000B00018951895189518951895189518951895D8
:1000C00018951895189518951895189518951895C8
:1000D00018951895189518951895189518951895B8
:1000E00018951895189518951895189518951895A8
:1000F0001895189518951895189518951895189598
:100100001895189518951895189518951895189587
:100110001895189518951895189518950C94BA086F
:100120001895189518951895189518951895189567
:10013000189518950C943A081895189518951895CF
:100140001895189518951895189518951895189547
:100150001895189518951895189518951895189537
:100160001895189518951895189518951895189527
:1001700018951895189518957F1BF63E7F1BF6BEAF
:1001800083E3D23E83E3D2BE0000803F16481E3D8B
:100190000000803FF671343E67FB64BD77C974BDD3
:1001A000F73E89BD3F6B84BECC32033ECABD273FBC
:1001B000CC32033E3F6B84BEF73E89BD77C974BD28
:1001C00067FB64BDE5FF3CBE6A8B31BED6704CBC9C
:1001D0000186593E0595A33E0186593ED6704CBC1A
:1001E0006A8B31BEE5FF3CBE0000B01B0D00AE17B0
:1001F000E918091934198D19D8190C1A431A7E1ADD
:10020000C91AFB1A351B741B0000F8200D00391F9A
:10021000721F871F9C1FC51F2E20592080209120F0
:10022000A220C020DA20EB200000CF220D000E21FA
:100230004D2162217721A02105222E225322642202
:1002400075229722B122C2220001282925294518AA
:10025000290218291182280B472801A028011829F2
:1002600001182901182902A0280534280175280140
:100270008228035028028228037E28FB03E333D020
:1002800000E117E228D100E117E225D100E117E2F1
:1002900022D103E328D000E117E21DD103E323D0EC
:1002A00008EE13E018D102E01ED008EE13E013D1DF
:1002B00008E019D008EE13E00ED101E014D000E1FF
:1002C00017E209D100E117E206D100E117E203D1FC
:1002D00006E009D008EE13E0FED00CE004D008EEF2
:1002E00013E0F9D008958A93802FE4E4F6E00081CA
:1002F0000F7B008302E310E0EED000916406007FE4
:1003000000936406082F02950F7010916406102B5D
:1003100010936406E4E4F6E000810068008302E3E1
:1003200010E0D9D0E4E4F6E000810F7700830AEF13
:1003300010E0D1D000916406007F009364068F70B6
:1003400000916406082B00936406E4E4F6E0008163
:100350000068008302E310E0BED0E4E4F6E0008130
:100360000F7700830AEF10E0B6D0899108958A9341
:10037000802FE4E4F6E000810064008302E310E0F3
:10038000AAD000916406007F00936406082F0295AE
:100390000F7010916406102B10936406E4E4F6E0ED
:1003A00000810068008302E310E095D0E4E4F6E009
:1003B00000810F7700830AEF10E08DD00091640672
:1003C000007F009364068F7000916406082B0093F1
:1003D0006406E4E4F6E000810068008302E310E0D4
:1003E0007AD0E4E4F6E000810F7700830AEF10E0B2
:1003F00072D0899108950E94E026C801A0E007C04C
:10040000B0E0FC01EA0FFB1F0081B1DFA395B0E073
:10041000FC01EA0FFB1F0081002311F0A13180F3E2
:10042000E4E00C94F1265FDF02E614E2E4DF0895D5
:100430000BEC0093520008E000935000E1E5F0E07F
:10044000008103FFFBCF03EC00935500E0E5F0E0F3
:10045000008100610083E1E5F0E0008104FFFBCF53
:1004600008ED04BF04E000934000E0E5F0E0008107
:100470000E7F0083089500E00093010200E20093E4
:10048000020203E00093040201E00093200200E274
:1004900000932102E0E0F2E0008101600083089512
:1004A00001E00093280200E300932902089501E08F
:1004B0000093300208E300933102089500E40093B2
:1004C000210300E5009324030DE00093200300E0E6
:1004D0000093220308950150104098018901232BB5
:1004E000D1F708958A93802F03C008EE1DEF07D03F
:1004F0008A95082F802F0023C1F789910895015014
:10050000104098018901232BD1F708950E94DC2621
:10051000942F81E035C0482F50E0440F551F440F01
:10052000551FFA01EA58FB4D00801180228033806C
:10053000482F50E0440F551F440F551FFA01E6584D
:10054000FB4D0082118222823382482F50E0440FFB
:10055000551F440F551FFA01E259FB4D00801180D1
:1005600022803380482F50E0440F551F440F551F01
:10057000FA01EE58FB4D00821182228233828A9565
:10058000813048F6EAE7F4E2008311832283338363
:10059000492F50E008E010E00E94AF23F801E05935
:1005A000FE4F4591559165917491EAE7F4E200811F
:1005B0001181228133810E946425E2E7F4E2008305
:1005C00011832283338381E061C0E0E7F1E0082FEB
:1005D00010E0000F111F000F111FE00FF11F492F36
:1005E00050E008E010E00E94AF23E00FF11F4591BA
:1005F000559165917491082F10E0000F111F000FA5
:10060000111FF801E658FB4D0081118122813381D1
:100610000E94642528013901E0E8F1E0082F10E08C
:10062000000F111F000F111FE00FF11F492F50E0A5
:1006300008E010E00E94AF23E00FF11F45915591B3
:1006400065917491082F10E0000F111F000F111F0A
:10065000F801EE58FB4D00811181228133810E9407
:100660006425A801B901820193010E944725E2E7B0
:10067000F4E240815181628173810E940325E2E7A7
:10068000F4E200831183228333838395823008F45C
:100690009CCFE2E7F4E20081118122813381E8E01E
:1006A0000C94ED260E94DC26942F81E035C0482F63
:1006B00050E0440F551F440F551FFA01EA57FB4DF8
:1006C0000080118022803380482F50E0440F551F56
:1006D000440F551FFA01E657FB4D0082118222821A
:1006E0003382482F50E0440F551F440F551FFA0125
:1006F000E258FB4D0080118022803380482F50E06B
:10070000440F551F440F551FFA01EE57FB4D008251
:100710001182228233828A95813048F6EAE8F4E237
:100720000083118322833383492F50E008E010E0D7
:100730000E94AF23F801E059FE4F45915591659114
:100740007491EAE8F4E200811181228133810E94F0
:100750006425E2E8F4E2008311832283338381E09D
:1007600061C0E0E7F1E0082F10E0000F111F000F5B
:10077000111FE00FF11F492F50E008E010E00E9428
:10078000AF23E00FF11F4591559165917491082FAA
:1007900010E0000F111F000F111FF801E657FB4D6D
:1007A00000811181228133810E9464252801390151
:1007B000E0E8F1E0082F10E0000F111F000F111FFB
:1007C000E00FF11F492F50E008E010E00E94AF2336
:1007D000E00FF11F4591559165917491082F10E03C
:1007E000000F111F000F111FF801EE57FB4D008184
:1007F0001181228133810E946425A801B9018201FF
:1008000093010E944725E2E8F4E240815181628130
:1008100073810E940325E2E8F4E2008311832283BE
:1008200033838395823008F49CCFE2E8F4E20081C0
:10083000118122813381E8E00C94ED260E94DC26B0
:10084000942F81E035C0482F50E0440F551F440FCE
:10085000551FFA01EA56FB4D00801180228033803B
:10086000482F50E0440F551F440F551FFA01E6561C
:10087000FB4D0082118222823382482F50E0440FC8
:10088000551F440F551FFA01E257FB4D00801180A0
:1008900022803380482F50E0440F551F440F551FCE
:1008A000FA01EE56FB4D00821182228233828A9534
:1008B000813048F6EAE9F4E200831183228333832E
:1008C000492F50E008E010E00E94AF23F801E05902
:1008D000FE4F4591559165917491EAE9F4E20081EA
:1008E0001181228133810E946425E2E9F4E20083D0
:1008F00011832283338381E061C0E0E7F1E0082FB8
:1009000010E0000F111F000F111FE00FF11F492F02
:1009100050E008E010E00E94AF23E00FF11F459186
:10092000559165917491082F10E0000F111F000F71
:10093000111FF801E656FB4D0081118122813381A0
:100940000E94642528013901E0E8F1E0082F10E059
:10095000000F111F000F111FE00FF11F492F50E072
:1009600008E010E00E94AF23E00FF11F4591559180
:1009700065917491082F10E0000F111F000F111FD7
:10098000F801EE56FB4D00811181228133810E94D6
:100990006425A801B901820193010E944725E2E97B
:1009A000F4E240815181628173810E940325E2E972
:1009B000F4E200831183228333838395823008F429
:1009C0009CCFE2E9F4E20081118122813381E8E0E9
:1009D0000C94ED260E94DE26542E80E090E0A0E0EC
:1009E000B0E04AE0442E1BC0442D50E0440F551F98
:1009F000440F551FFA01E256FB4D00801180228002
:100A00003380442D50E0440F551F440F551FFA0109
:100A1000EE55FB4D00821182228233824A9441E0DE
:100A2000441610F7E2EAF4E2008311832283338351
:100A300044242CC0ECE6F1E0042D10E0000F111F5F
:100A4000000F111FE00FF11F452D50E00CE210E0E8
:100A50000E94AF23E00FF11F45915591659174916C
:100A6000042D10E0000F111F000F111FF801EE55AB
:100A7000FB4D00811181228133810E946425AC01EC
:100A8000BD010E940325C801D90143940BE0401623
:100A900088F28C019D01E6E00C94EF260E94DE2690
:100AA000542E80E090E0A0E0B0E04AE0442E1BC06D
:100AB000442D50E0440F551F440F551FFA01E653D3
:100AC000FB4D0080118022803380442D50E0440F84
:100AD000551F440F551FFA01E253FB4D008211824E
:100AE000228233824A9441E0441610F7EEECF4E29D
:100AF000008311832283338344242CC0ECE6F1E08D
:100B0000042D10E0000F111F000F111FE00FF11F47
:100B1000452D50E00CE210E00E94AF23E00FF11FE2
:100B20004591559165917491042D10E0000F111FAE
:100B3000000F111FF801E253FB4D0081118122814A
:100B400033810E946425AC01BD010E940325C801C8
:100B5000D90143940BE0401688F28C019D01E6E038
:100B60000C94EF260E94DE26542E80E090E0A0E058
:100B7000B0E04AE0442E1BC0442D50E0440F551F06
:100B8000440F551FFA01EA50FB4D0080118022806E
:100B90003380442D50E0440F551F440F551FFA0178
:100BA000E650FB4D00821182228233824A9441E05A
:100BB000441610F7EAEFF4E20083118322833383B3
:100BC00044242CC0ECE6F1E0042D10E0000F111FCE
:100BD000000F111FE00FF11F452D50E00CE210E057
:100BE0000E94AF23E00FF11F4591559165917491DB
:100BF000042D10E0000F111F000F111FF801E65027
:100C0000FB4D00811181228133810E946425AC015A
:100C1000BD010E940325C801D90143940BE0401691
:100C200088F28C019D01E6E00C94EF260E94DE26FE
:100C3000542E80E090E0A0E0B0E048E0442E1BC0DD
:100C4000442D50E0440F551F440F551FFA01EE5D2F
:100C5000FA4D0080118022803380442D50E0440FF3
:100C6000551F440F551FFA01EA5DFA4D00821182AB
:100C7000228233824A9441E0441610F7E6E2F5E21C
:100C8000008311832283338344242CC0E0EAF1E003
:100C9000042D10E0000F111F000F111FE00FF11FB6
:100CA000452D50E004E210E00E94AF23E00FF11F59
:100CB0004591559165917491042D10E0000F111F1D
:100CC000000F111FF801EA5DFA4D008111812281A8
:100CD00033810E946425AC01BD010E940325C80137
:100CE000D901439409E0401688F28C019D01E6E0A9
:100CF0000C94EF260E94DE26542E80E090E0A0E0C7
:100D0000B0E048E0442E1BC0442D50E0440F551F76
:100D1000440F551FFA01EA5BFA4D008011802280D2
:100D20003380442D50E0440F551F440F551FFA01E6
:100D3000E65BFA4D00821182228233824A9441E0BE
:100D4000441610F7EAE4F5E200831183228333832B
:100D500044242CC0E0EAF1E0042D10E0000F111F44
:100D6000000F111FE00FF11F452D50E004E210E0CD
:100D70000E94AF23E00FF11F459155916591749149
:100D8000042D10E0000F111F000F111FF801E65B8A
:100D9000FA4D00811181228133810E946425AC01CA
:100DA000BD010E940325C801D901439409E0401602
:100DB00088F28C019D01E6E00C94EF260E94DE266D
:100DC000542E80E090E0A0E0B0E048E0442E1BC04C
:100DD000442D50E0440F551F440F551FFA01E659AA
:100DE000FA4D0080118022803380442D50E0440F62
:100DF000551F440F551FFA01E259FA4D0082118226
:100E0000228233824A9441E0441610F7EEE6F5E27E
:100E1000008311832283338344242CC0E0EAF1E071
:100E2000042D10E0000F111F000F111FE00FF11F24
:100E3000452D50E004E210E00E94AF23E00FF11FC7
:100E40004591559165917491042D10E0000F111F8B
:100E5000000F111FF801E259FA4D00811181228122
:100E600033810E946425AC01BD010E940325C801A5
:100E7000D901439409E0401688F28C019D01E6E017
:100E80000C94EF260E94DC26842FA52F0E94A42418
:100E9000482F50E0440F551F440F551FFA01EE56DE
:100EA000FA4D40815181628173810E94472528015A
:100EB00039010A2F10E020E030E00E94AF24A801A1
:100EC000B901820193010E94DD25482F50E0440FB3
:100ED000551F440F551FFA01EE56FA4D40815181BE
:100EE000628173810E94032590E0880F991F880F0B
:100EF000991FFC01EE56FA4D008311832283338340
:100F0000E8E00C94ED261091480001E000934800C1
:100F10002091A0003091A2000091A2000C7F0460FB
:100F20000093A2004FB77894E8E4F0E000810160FC
:100F300000835091CD01EF93FF930F932F93EBEC30
:100F4000F1E008ED21E004BF20832F910F91FF9184
:100F5000EF9103E00093CD01889510934800209312
:100F6000A0003093A2005093CD014FBF0895EFEC45
:100F7000F1E0008107FDFBCF0895F9DFEFECF1E030
:100F8000008101FF11C006E30093CA01EF93FF93B4
:100F90000F932F93EBECF1E008ED21E004BF2083E9
:100FA0002F910F91FF91EF9108959A938A93C80121
:100FB000DEDF8B3000E0900748F04091D22750E010
:100FC00000E410E00E94AF23800F911F082F0093D0
:100FD000C001892F8F718093C10100E00093C2018D
:100FE00006E00093CA01EF93FF930F932F93EBEC6E
:100FF000F1E008ED21E004BF20832F910F91FF91D4
:10100000EF910091C4018991999108950E94E12680
:10101000C801A22F00E00093060900E000934608F3
:101020008B3000E0900748F04091D22750E000E478
:1010300010E00E94AF23800F911F9FDF03E3009316
:10104000CA01082F0093C001892F8F718093C101BD
:1010500000E00093C201A093C40105E30093CA011C
:1010600052DF03E00093060901E000934608E3E045
:101070000C94F2269A938A93FA93EA930A927A93BB
:101080006A935A934A933A932A931A930A930FB600
:10109000E0E0F2E00081046000830091AD27039559
:1010A0000F700093AD270091B027002399F10091B4
:1010B000322710913327212F220F220B322F4091FC
:1010C000AD2750E0440F551F440F551FFA01EE5253
:1010D000F94D4081518162817381400F511F621F20
:1010E000731F408351836283738380914227909161
:1010F000432701968093422790934327803008E04E
:10110000900741F400E00093B02710E000934227DD
:10111000109343270091AD2710E0000F111FF80135
:10112000EE52FA4D00811181009338031093390378
:10113000E5E2F3E0008101FF0EC00091AD2710E071
:10114000000F111FF801EE50FA4D0081118100933C
:101150003A0310933B030FBE0991199129913991DC
:1011600049915991699179910990E991F991899100
:10117000999118954A933A932A931A930A934FB7E1
:1011800000911002109111022091CC273091CD27AF
:10119000021B130B00933227109333274FBF099183
:1011A000199129913991499118957A926A925A9296
:1011B0004A929A938A93FA93EA933A922A921A92CB
:1011C0000A927A936A935A934A933A932A931A9378
:1011D0000A939FB70091B027002309F050C30091F4
:1011E000B627002321F408E00093C52703C004E0DC
:1011F0000093C52780E033C05091C527482F642F46
:10120000082F10E0000F111F000F111FF801EE5200
:10121000F94D008111812281338142E00E9417241F
:10122000462F30DE0E94B124282F30E0220F331FDA
:10123000F901EE5EF84D0083118300E010E020E03C
:1012400030E0482F50E0440F551F440F551FFA015E
:10125000EE52F94D008311832283338383958031CD
:1012600058F20FEF0093B02700E010E020E030E0EC
:10127000ECE4F7E20083118322833383E8E4F7E2AE
:101280000083118322833383E4E4F7E20083118334
:101290002283338300E010E020E030E0EEECF7E260
:1012A000008311832283338380E0CFC0082F10E0B6
:1012B000000F111FF801EE5EF84D00811181212F02
:1012C000220F220B322F0E94A42428013901082F5B
:1012D00010E0000F111FF801EE5EF84D0081118142
:1012E000212F220F220B322F0E94A424A201B3012E
:1012F0000E946425EEECF7E24081518162817381A6
:101300000E940325EEECF7E20083118322833383EE
:10131000E4E4F7E200811181228133810E94A42458
:1013200028013901082F10E0000F111FF801EE5EAF
:10133000F84D00811181212F220F220B322F0E94A4
:10134000A424482F50E0440F551F440F551FFA01A5
:10135000EE5EF94D40815181628173810E94642566
:10136000A201B3010E9403250E94B124E4E4F7E244
:101370000083118322833383E8E4F7E20081118143
:10138000228133810E94A42428013901082F10E012
:10139000000F111FF801EE5EF84D00811181212F21
:1013A000220F220B322F0E94A424482F50E0440F1A
:1013B000551F440F551FFA01EE5AF94D40815181D6
:1013C000628173810E946425A201B3010E940325FA
:1013D0000E94B124E8E4F7E200831183228333837F
:1013E000ECE4F7E200811181228133810E94A42480
:1013F00028013901082F10E0000F111FF801EE5EDF
:10140000F84D00811181212F220F220B322F0E94D3
:10141000A424482F50E0440F551F440F551FFA01D4
:10142000EE56F94D40815181628173810E9464259D
:10143000A201B3010E9403250E94B124ECE4F7E26B
:1014400000831183228333838395803108F42ECF68
:1014500040E050E060E871E4EEECF7E200811181D9
:10146000228133810E94DD250E94482BEEECF7E2B9
:101470000083118322833383EEECF7E20081118134
:10148000228133810E94B12440E150E00E94DB239D
:101490000093CA271093CB27E4E4F7E2008111817F
:1014A00022813381E8E5F7E20083118322833383CD
:1014B000E8E4F7E20081118122813381ECE5F7E273
:1014C0000083118322833383ECE4F7E200811181EE
:1014D00022813381E4E6F7E20083118322833383A0
:1014E0000091AF27002339F100E00093AF27E8E532
:1014F000F7E20081118122813381ECE6F7E200837B
:10150000118322833383ECE5F7E20081118122818C
:101510003381E8E6F7E20083118322833383E4E634
:10152000F7E20081118122813381E0E7F7E2008355
:10153000118322833383ECE6F7E20081118122815B
:101540003381E8E5F7E24081518162817381401B7C
:10155000510B620B730B4083518362837383E8E604
:10156000F7E20081118122813381ECE5F7E24081CD
:10157000518162817381401B510B620B730B40835D
:10158000518362837383E0E7F7E200811181228156
:101590003381E4E6F7E24081518162817381401B2F
:1015A000510B620B730B40835183628373830091F1
:1015B000B627002309F0B4C00091C3270130C9F554
:1015C00041E0E8E5F7E200811181228133810E9448
:1015D000A4240E9486020E94B124E0E9F7E200837D
:1015E00011832283338341E0ECE5F7E2008111812E
:1015F000228133810E94A4240E9452030E94B124BC
:10160000E4E9F7E2008311832283338341E0E4E6D7
:10161000F7E200811181228133810E94A4240ED936
:101620000E94B124ECE8F7E2008311832283338324
:101630009BC00091C3270230B9F541E0E8E5F7E22D
:1016400000811181228133810E94A424EFDA0E945B
:10165000B124E0E9F7E2008311832283338341E080
:10166000ECE5F7E200811181228133810E94A424FC
:1016700041DB0E94B124E4E9F7E200831183228375
:10168000338341E0E4E6F7E2008111812281338176
:101690000E94A42493DB0E94B124ECE8F7E20083CB
:1016A00011832283338360C00091C327033009F084
:1016B0005BC041E0E8E5F7E20081118122813381DE
:1016C0000E94A42487D90E94B124E0E9F7E20083B4
:1016D00011832283338341E0ECE5F7E2008111813D
:1016E000228133810E94A424D9D90E94B124E4E943
:1016F000F7E2008311832283338341E0E4E6F7E2DB
:1017000000811181228133810E94A4242BDA0E945E
:10171000B124ECE8F7E2008311832283338324C0F1
:10172000E8E5F7E20081118122813381E0E9F7E207
:101730000083118322833383ECE5F7E2008111817A
:1017400022813381E4E9F7E200831183228333832A
:10175000E4E6F7E20081118122813381ECE8F7E2CF
:1017600000831183228333830091BF270095009368
:10177000BF270091BF27002309F05CC084E00091DF
:10178000C627801BE0E9F7E20081118122813381C5
:10179000ECE9F7E24081518162817381040F151FEA
:1017A000261F371F482F50E060E070E00E9442245F
:1017B000E0E5F7E20083118322833383E4E9F7E273
:1017C0000081118122813381E0EAF7E24081518179
:1017D00062817381040F151F261F371F482F50E0A9
:1017E00060E070E00E944224E4E5F7E200831183A8
:1017F00022833383ECE8F7E2008111812281338177
:10180000E8E9F7E24081518162817381040F151F7D
:10181000261F371F482F50E060E070E00E944224EE
:10182000E0E6F7E200831183228333830FEF009316
:10183000C0272BC0E0E9F7E20081118122813381CA
:10184000ECE9F7E20083118322833383E4E9F7E2D2
:101850000081118122813381E0EAF7E20083118364
:1018600022833383ECE8F7E2008111812281338106
:10187000E8E9F7E2008311832283338306C008E29C
:1018800010E000936608109367089FBF09911991B3
:1018900029913991499159916991799109901990BA
:1018A00029903990E991F9918991999149905990AC
:1018B0006990799018950E94E02600E40E947301D7
:1018C000AFEF80E002C0A69583958830A8F4BA2FC8
:1018D00090E005C000E00E94B701B695939598305E
:1018E00090F7BB2311F001E001C000E0002391F765
:1018F0000FE10E94B701F1CFE4E00C94F1260E94C1
:10190000E026D80180E090E02FC006E110E0AC01B5
:101910000E94AF230A0F1B1F212F220F220B322FF1
:101920000E94A42440E050E064EB73E40E947E2611
:1019300030F440E050E064EB73EC0E94032545E393
:101940005AEF6EE87CE30E9464250E945D23AC019F
:10195000440F551F440F551FFA01EE56F94D0083F1
:101960001183228333830196803100E090076CF26B
:10197000E4E00C94F1260E94E026D80180E090E09B
:101980002FC006E110E0AC010E94AF230A0F1B1F1D
:10199000212F220F220B322F0E94A42440E050E07E
:1019A00064EB73E40E947E2630F440E050E064EB88
:1019B00073EC0E94032545E35AEF6EE87CE30E9436
:1019C00064250E947A2AAC01440F551F440F551F0D
:1019D000FA01EE5EF94D0083118322833383019671
:1019E000803100E090076CF2E4E00C94F1260E9454
:1019F000E026D80180E090E02FC006E110E0AC01C5
:101A00000E94AF230A0F1B1F212F220F220B322F00
:101A10000E94A42440E050E064EB73E40E947E2620
:101A200030F440E050E064EB73EC0E94032545E3A2
:101A30005AEF6EE87CE30E9464250E945D23AC01AE
:101A4000440F551F440F551FFA01EE5AF94D0083FC
:101A50001183228333830196803100E090076CF27A
:101A6000E4E00C94F1260E94DC26D80180E090E0AE
:101A700034C08D01212F220F220B322F0E94A4246B
:101A8000280139018C01212F220F220B322F0E94B5
:101A9000A42449E058E964EC7EE30E9464250E9496
:101AA0007A2AA201B3010E946425280139018D011F
:101AB000212F220F220B322F0E94A424A201B30156
:101AC0000E9403250E94B1249C01220F331FF901BB
:101AD000EE50FA4D008311830196803100E09007AB
:101AE00044F2E8E00C94ED260E94DA264801D90180
:101AF00080E090E046C006E110E0AC010E94AF2318
:101B0000A801480D591D483601E0500714F0485609
:101B100051408D01212F220F220B322F0E94A4242D
:101B2000280139018A01212F220F220B322F0E9416
:101B3000A4240801190145E35AEF6EE87CE3800113
:101B400091010E9464250E947A2AA201B3010E9499
:101B50006425280139018D01212F220F220B322FFC
:101B60000E94A424A201B3010E9403250E94B12473
:101B70009C01220F331FF901EE52FA4D00831183AD
:101B80000196803100E090070CF4B5CFEAE00C94A8
:101B9000EB260E94E0262091AB273091AC270091E4
:101BA000A9271091AA27A0DF4CD106E00E9472025B
:101BB000E091CA27F091CB27F3970CF4F1C080E0B5
:101BC0009CE5A1ECB7E400E010E00093D727109368
:101BD000D82708C0E7EDF7E200811181065F1F4FAB
:101BE000008311830091D7271091D827083621E070
:101BF0001207BCF520910824309109240091D727C1
:101C00001091D82771DF04E00E9472020091CA2768
:101C10001091CB27212F220F220B322F0E94A424B8
:101C2000AC01BD010E946626A8F60091CA2710915A
:101C3000CB27212F220F220B322F0E94A424C80170
:101C4000D9010091D7271091D8270093D32710935B
:101C5000D427E091CA27F091CB27B8970CF0BACFE0
:101C600054C080E09CE5A1ECB7E40AE010E0ADD000
:101C700000E010E0009308241093092408C0E8E075
:101C8000F4E200811181025E1F4F008311830091F5
:101C9000082410910924083E27E01207B4F520918A
:101CA0000824309109240091D3271091D4271CDFF8
:101CB00004E00E9472020091CA271091CB27212FC5
:101CC000220F220B322F0E94A424AC01BD010E94DE
:101CD0006626A8F60091CA271091CB27212F220F44
:101CE000220B322F0E94A424C801D901009108249C
:101CF000109109240093D5271093D627E091CA2785
:101D0000F091CB2774970CF0BACFE091D327F091E4
:101D1000D4273B9744F0E3EDF7E2008111810850AE
:101D2000104000831183E091D527F091D627759755
:101D300044F0E5EDF7E2008111810F50104000837F
:101D400011832091D5273091D6270091D327109168
:101D5000D427CADE0091D5271091D6270093AB2750
:101D60001093AC270091D3271091D4270093A92773
:101D70001093AA273091AA27232F00E210E046D91A
:101D80002091A92701E210E041D93091AC27232FFF
:101D900002E210E03BD92091AB2703E210E036D9F4
:101DA0000FEF0093AE27E4E00C94F12634E030937B
:101DB00040093091C127329F00926A0910926B0945
:101DC0000093660910936709089524E044E650E003
:101DD0000E94AF23EBDF48E750E0009136271091D7
:101DE00037270E94DB2303950E94720200E00093D4
:101DF000400908958A93812F10E0E7DF00E513EC96
:101E00000E947F02082F10E0E0DF899108950E9470
:101E1000E026D80181E090E00DC042E050E08C0166
:101E20000E94DB23202F8D01C1DF00E513EC0E940F
:101E30007F020196843100E090077CF3E4E00C948B
:101E4000F12620E231E202E614E20E942D2B00E8A6
:101E50000E94130200E310E0B8DF08950E94F5220B
:101E600040E050E064E672E40E9464250E94B124E0
:101E700008950E94DC26D80121E331E202E614E253
:101E80000E942D2B00E80E941302A13000E0B00751
:101E900014F180E0082F10E020E030E00E94AF2431
:101EA000280139018D01212F220F220B322F0E9490
:101EB000A4240E94FA26A801B901820193010E947C
:101EC000662678F5082F07570E9473010EE30E94DB
:101ED000B7018395DFCF80E008C006E8081B0E94A9
:101EE00073010CE30E94B7018395082F10E020E0F6
:101EF00030E00E94AF24280139010FEF1FEFAD0140
:101F00000E94AF23212F220F220B322F0E94A424E4
:101F10000E94FA26A801B901820193010E94662657
:101F2000E0F200E315E70E947F02E8E00C94ED2662
:101F30009A938A9300E010E080E090E019C0E0E01E
:101F4000F2E020812860208320912B022223E1F3FC
:101F500021E020932B022091120230911302020FF4
:101F6000131F095B1040112312F400E010E00196EA
:101F7000803A20E092071CF34DE450E00E94DB23FE
:101F8000899199910895E0E0F2E000810061008379
:101F9000009133020023E1F301E00093330240910A
:101FA000BC2750E000911402109115020E94C32337
:101FB00008950091A5271091A627DDDC0091A527A3
:101FC0001091A62714DD0091A5271091A627009354
:101FD000A7271093A8270091A7271091A8278FDC87
:101FE00008950091A5271091A627C5DC0091A5278B
:101FF0001091A627FCDC0091A7271091A8277FDC71
:10200000009136271091372700932609109327094E
:102010004091C72750E00FEF10E00E94AF2323DD6F
:1020200008959A938A9300E110E00E94D507902FBB
:1020300080E001E110E00E94D50710E0802B912B99
:10204000809336279093372706E110E00E94D5074A
:10205000902F80E007E110E00E94D50710E0802B70
:10206000912B8093A5279093A62708E110E00E946A
:10207000D507902F80E009E110E00E94D50710E01D
:10208000802B912B8093A7279093A82700E210E044
:102090000E94D507902F80E001E210E00E94D50752
:1020A00010E0802B912B8093A9279093AA2702E21E
:1020B00010E00E94D507902F80E003E210E00E941C
:1020C000D50710E0802B912B8093AB279093AC2702
:1020D00002E110E00E94D5070093B92703E110E068
:1020E0000E94D5070093BA2705E110E00E94D507AA
:1020F0000093BB2704E210E00E94D5070093C42799
:102100000EE110E00E94D5070093C7270FE110E011
:102110000E94D5070093C32709E010E00E94D5076D
:102120000093BD270AE010E00E94D5070093BC276A
:1021300005E210E00E94D5070093C1270BE010E0F4
:102140000E94D5070093C22707E210E00E94D5073E
:1021500003700093C6270CE110E00E94D507802F82
:1021600090E00DE110E00E94D507102F00E0802BD9
:10217000912B8093C8279093C927E8ECF7E2008160
:1021800011810160106800831183899199910895EC
:102190000E94D4262497F8940E941802E0E8F6E002
:1021A000008108600083009160060F600093600664
:1021B00000914006006C00934006E0E6F6E00081E6
:1021C00000620083E0E4F6E0008102600083009199
:1021D0006006006C0093600608E10093110608E1B8
:1021E0000093120608E10093130608E100933006FD
:1021F0000E943E0160DB08E010E00E94D5070F3F1F
:1022000011F401E001C000E0E8E0F6E0108111FD0A
:1022100009C0E8E0F6E0108112FD02C011E003C041
:1022200010E001C010E0012B002309F49EC000E083
:102230000093D2270FC02AE20A2F10E0085D1F4F3B
:102240000E940608A395AB30B0F30091D227039506
:102250000093D2270091D227043008F081C022E4F5
:1022600031E202E614E20E942D2B00E80E941302E4
:1022700008E20E94720221E000E110E00E940608DC
:1022800026E701E110E00E94060820E006E110E0E8
:102290000E94060828E207E110E00E94060820E0FC
:1022A00008E110E00E94060828E209E110E00E941F
:1022B000060820E000E210E00E94060820E001E2AB
:1022C00010E00E94060820E002E210E00E940608EA
:1022D00020E003E210E00E94060822E002E110E0A4
:1022E0000E94060828E003E110E00E94060820E0B2
:1022F00005E110E00E94060825E00EE110E00E94D2
:10230000060822E00FE110E00E94060821E004E246
:1023100010E00E94060820E00CE110E00E94060890
:1023200020E00DE110E00E94060828EC09E010E032
:102330000E94060824E30AE010E00E94060824E058
:1023400005E210E00E94060824E00BE010E00E9485
:10235000060822E007E210E00E940608A0E073CF22
:1023600020E008E010E00E94060808E010E00E946B
:10237000D5070093D22755DE08E00093BA2702E084
:102380000093B92701E00093C32703E200930108FB
:1023900007E00093000806E910E000932608109378
:1023A00027080091C22710E000932A0810932B08F9
:1023B00007E00093400809EA13E0009366081093D1
:1023C000670801E00093460801E0009300090091CE
:1023D000362710913727009326091093270903E029
:1023E000009306090091A20007600093A2000E94DA
:1023F0005E022091AB273091AC270091A927109164
:10240000AA2772DB04E414E000930C0210930D027F
:102410000E943B0202E0009322020E9457020E94A7
:102420005002DFDD02E00E94720203E200934109E4
:10243000009164060F730093640622E531E202E620
:1024400014E20E942D2B00EC0E94130223E631E2DD
:1024500002E614E20E942D2B00E80E94130200ED18
:1024600017E0D5DC00EA1FE0D2DC00E41FE1CFDC9E
:1024700000ED17E0CCDC00E00093400900E00093A1
:10248000400900E50E947202009163240B3469F652
:1024900000916424003549F6009165240F3429F633
:1024A00000916406006C009364060091BD2710E063
:1024B000005A164F0093CC271093CD270091672424
:1024C000023309F0B2CF789424E731E202E614E255
:1024D0000E942D2B00EC0E941302AEE10A2FA02FC8
:1024E000AA95002309F4C5C00091D22710E01A93E1
:1024F0000A9325E831E202E614E20E942D2B22968F
:1025000000E80E94130206E00E947202E8E0F6E092
:10251000008102FD17C00091D22703950093D227B6
:10252000033018F002E00093D2272091D22708E070
:1025300010E00E94060802E310E047DC72DD51DD86
:10254000A4E11BC0E8E0F6E0008101FD16C00091A7
:10255000D2270A950093D2270F3F19F400E0009389
:10256000D2272091D22708E010E00E94060802E35B
:1025700010E02BDC56DD35DDA4E102EC0E94730196
:10258000CC2409C00C2D10E0085D1F4F0E94D50718
:102590000E94B701C3940BE0C016A0F3E8E0F6E098
:1025A000008103FD9BCF08E210E00FDC0DE00E94EC
:1025B0007301A0E402E00093BE270EC00091BE2785
:1025C00003950093BE270D3018F00CE00093BE2752
:1025D000A0E408E210E0F9DB0091BE2700540E945D
:1025E000730105E00E947202E8E0F6E0008102FF5C
:1025F000E5CFE8E0F6E0008101FD0FC00091BE27C5
:102600000A950093BE27023018F402E00093BE271B
:10261000A0E408E210E0D9DBDFCFE8E2F6E00081D9
:1026200000FD1AC0A3950A2FA02F0B3508F0A0E3D8
:102630000A2F0E94B7010091BE2700540E94730127
:1026400002E310E0C2DB2A2F0091BE2710E00A5DF2
:102650001F4F0E940608C0CFE8E0F6E0008103FDAE
:10266000BBCF0091BE27033008F4B6CF08E210E0DC
:10267000ACDB0CE00E94730100E310E0A6DBA4E1F8
:102680004FC0E8E2F6E0008100FD04C000E310E086
:102690009CDBA4E64DDC380140913627509137276A
:1026A0004F5F5F4F652F660F660B762F00E01CE6CD
:1026B0002CED32E00E94422444E00E941724C8011D
:1026C0007A926A929A938A9327E931E202E614E2B7
:1026D0000E942D2B249600E80E9413020091CA2725
:1026E0001091CB271A930A9327EA31E202E614E20B
:1026F0000E942D2B229600EC0E9413020091C62707
:1027000010E01A930A9323EB31E202E614E20E94EE
:102710002D2B22960AEC0E94130202E00E94720204
:102720000A2FA02FAA95002309F0ABCF0AE060166C
:1027300000E07006ACF42CEB31E202E614E20E94F9
:102740002D2B00E80E94130200ED10E03EDB00EBB1
:1027500010E03BDB00ED10E038DB02E10E9472028A
:102760000091CA271091CB27093E23E01207ACF055
:102770002DEC31E202E614E20E942D2B00EC0E94C7
:10278000130200ED10E021DB00EB10E01EDB00ED9A
:1027900010E01BDB04E10E9472020AE00E94720258
:1027A00001E00093AF2700E00093BE270EEF0983FE
:1027B00000E0088306E00093B72700E010E00093F4
:1027C0003C2710933D2700933A2710933B27212F56
:1027D000220F220B322FE0E6F7E2008311832283DF
:1027E0003383FF24EE24E39404E10E94720200E3A9
:1027F00010E0EBDA03E00E94720200E310E0E5DA99
:102800001CC000916406006C0093640600E2009313
:10281000A427C3940C2DC02E053678F0CC2400E0FC
:102820000093400900E010E0009338271093392707
:10283000EE24FF2401E00093AF270091B42700238A
:1028400009F077C30091B627002309F0C0C1E0E585
:10285000F7E20081118122813381E4E7F7E200830E
:10286000118322833383E4E5F7E200811181228121
:102870003381E0E8F7E20083118322833383E0E6CB
:10288000F7E20081118100933427109335270091DE
:10289000B92710E02091342730913527021713070C
:1028A0000CF061C10091B327002309F05CC1CC2476
:1028B00000E00093B7270091B82703950093B8274D
:1028C000E8E7F7E20081118122813381E4E7F7E252
:1028D0004081518162817381401B510B620B730BEC
:1028E0004083518362837383E4E8F7E200811181BE
:1028F00022813381E0E8F7E2408151816281738176
:10290000401B510B620B730B4083518362837383B3
:10291000E4E7F7E20081118122813381E4E7F7E205
:1029200040815181628173810E94EF2348015901E6
:10293000E0E8F7E20081118122813381E0E8F7E2EB
:1029400040815181628173810E94EF23800E911E2C
:10295000A21EB31E840195010E94A4240E94482B4C
:102960000E94B12443E00E94BD232801552042F477
:1029700022E104EF1EE71ADA00E21EE40E947F0261
:10298000E0E8F7E200811181228133810E94A424D2
:10299000A801B9014A015B01E4E7F7E20081118176
:1029A000228133810E94A424A401B50157DA009347
:1029B000382710933927842D0091C127800F8395E4
:1029C0000A811B8120913427309135270217130784
:1029D0007CF4009138271091392700933E271093FB
:1029E0003F27720100913427109135270A831B83FA
:1029F000E0913E27F0913F273197E63500E0F00760
:102A000008F060C04AE050E0009138271091392763
:102A10000E94DB23402F4A5F0091C8271091C927ED
:102A20000E94BD230170002309F04CC000913E2795
:102A300010913F2700933C2710933D2700933827A0
:102A4000109339270091C427013029F4282F00E47E
:102A50001FE1ACD96EC20091C4270230E9F4E091C5
:102A60003827F091392775972CF4282F00EB16E3BF
:102A70009DD95FC20091382710913927063420E094
:102A800012072CF0282F00E717E190D952C2282F07
:102A900000E41FE18BD94DC2282FB22F8AE090E0CD
:102AA0004AE050E000913827109139270E94DB233B
:102AB000AC01401B510B00ED17E00E94AF232B2F00
:102AC00075D937C20091BA27002309F432C2109198
:102AD000392711230AF02DC20091BA2710E0209166
:102AE000342730913527021713070CF022C294E0E7
:102AF0004CEE5FEF00913827109139270E94DB23BD
:102B0000901B492F0091C8271091C9270E94BD230F
:102B10000170002309F00DC2009138271091392768
:102B200000933C2710933D270091C4270430B1F453
:102B3000282FB22F86E190E04AE050E0009138273C
:102B4000109139270E94DB23AC01401B510B08EE8A
:102B500013E00E94AF232B2F29D9EBC1282F00E9C6
:102B600015E624D9E6C100E010E000936A0910934D
:102B70006B0900E010E0009366091093670900E01C
:102B800000934009E4E7F7E200811181228133815B
:102B9000E8E7F7E20083118322833383E0E8F7E27A
:102BA0000081118122813381E4E8F7E200831183FF
:102BB0002283338300E010E00A831B830091B72750
:102BC00003950093B72700E00093B827B2C10091A6
:102BD000C327033009F0D0C042E050E060E070E06D
:102BE000E0E5F7E200811181228133810E944224D5
:102BF000E4E7F7E2008311832283338342E050E06D
:102C000060E070E0E4E5F7E2008111812281338128
:102C10000E944224E0E8F7E2008311832283338399
:102C200042E050E060E070E0E0E6F7E20081118110
:102C3000228133810E944224009334271093352748
:102C4000E4E7F7E20081118122813381E4E7F7E2D2
:102C500040815181628173810E94EF2348015901B3
:102C6000E0E8F7E20081118122813381E0E8F7E2B8
:102C700040815181628173810E94EF23800E911EF9
:102C8000A21EB31E840195010E94A4240E94482B19
:102C90000E94B12444E00E94BD232801552042F443
:102CA00022E100E01DE782D800E513EC0E947F02DC
:102CB000D3940D2DD02E053120F001E00093AF27E5
:102CC000DD240091B327002309F033C1009134279C
:102CD00010913527212F220F220B322F0E94A4247E
:102CE0000E94FA260E94B124802F889F802D42E006
:102CF0000091C1270E949123800FE0E8F7E2008154
:102D00001181228133810E94A424A801B9014A01C2
:102D10005B01E4E7F7E200811181228133810E94A7
:102D2000A424A401B5019AD800933C2710933D2711
:102D30000091C427013081F410913D27112332F016
:102D4000282F00E117E20E94D60E14C0282F00E2BF
:102D50001EE40E94D60E0EC0282F622F40EE5EE2C7
:102D6000E4E7F7E200811181401B510B8A01262F15
:102D70000E94D60E7201DDC042E050E060E070E0DB
:102D8000E0E5F7E200811181228133810E94422433
:102D9000E4E7F7E2008311832283338342E050E0CB
:102DA00060E070E0E4E5F7E2008111812281338187
:102DB0000E944224E0E8F7E20083118322833383F8
:102DC00042E050E060E070E0E0E6F7E2008111816F
:102DD000228133810E9442240093342710933527A7
:102DE000E4E7F7E20081118122813381E4E7F7E231
:102DF00040815181628173810E94EF234801590112
:102E0000E0E8F7E20081118122813381E0E8F7E216
:102E100040815181628173810E94EF23800E911E57
:102E2000A21EB31E840195010E94A4240E94482B77
:102E30000E94B12445E00E94BD2328010091B927DA
:102E400010E02091342730913527021713070CF03A
:102E500065C00091B327002309F060C00091B82736
:102E600003950093B827043631F401E00093AF27AF
:102E700000E00093B827CC2400E00093B72755204A
:102E80004AF422E100E01DE70E94D60E00E513ECB3
:102E90000E947F020091342710913527212F220FA5
:102EA000220B322F0E94A4240E94FA260E94B124F1
:102EB000802F889F802D42E00091C1270E9491239E
:102EC000800F0091B827033058F0282F00EE1EE243
:102ED0004091342750913527041B150B0E94D60EC4
:102EE0007201E0E8F7E200811181228133810E94C2
:102EF000A424A801B9014A015B01E4E7F7E20081DB
:102F00001181228133810E94A424A401B5010E9471
:102F10002E0F00933C2710933D270BC000E0009339
:102F2000400900E00093B8270091B727039500936C
:102F3000B7270091B727083C41F010E00091B8276F
:102F4000083C19F01060112319F001E00093AF273D
:102F50000091B327E8EEF1E00C948F2680913C2796
:102F600090913D2701E0E01600E0F0062CF0809300
:102F70003A2790933B2704C080913A2790913B27B2
:102F8000992352F09A938A932EED31E202E614E2ED
:102F90000E942D2B229609C09A938A9325EE31E246
:102FA00002E614E20E942D2B229600E80E941302F2
:102FB0000981102F13951983002371F4088100955E
:102FC00008830881002329F46090CA277090CB27DA
:102FD00003C00E94C30F38018701212F220F220B4B
:102FE000322F0E94A4240E94FA260E94B124C80114
:102FF00004E80E947301082F0E94B701992352F43C
:103000002BEE31E202E614E20E942D2B04E80E942E
:1030100013021EC00091A42710E01A930A93009196
:10302000C32710E01A930A930091B92710E01A936E
:103030000A930091BA2710E01A930A932DEE31E219
:1030400002E614E20E942D2B289605E80E94130246
:1030500008810023B1F04AE050E083010E94DB23A5
:103060005A934A934AE050E083010E94DB231A936B
:103070000A9329EF31E202E614E20E942D2B2496F6
:1030800009C07A926A9220E032E202E614E20E94DB
:103090002D2B22960CE80E9413020091B6270023E4
:1030A00009F04FC00091B727043048F024E731E21F
:1030B00002E614E20E942D2B00EC0E941302A82FBE
:1030C000A83008F0AFEFE0913827F0913927319719
:1030D0007CF00091382710913927045C1F4F4AE09B
:1030E00050E00E94DB23009340271093412712C039
:1030F00042E050E000913827109139270E94DB23ED
:103100000E5C1F4F4AE050E00E94DB2300934027F3
:10311000109341270091402700540E947301A23070
:1031200020F006E00E94B70105C0A13019F403E0C9
:103130000E94B70105EC0E9473010FE20E94B701E3
:103140000FC343E082010E94BD23C801833C01E01C
:10315000900734F400E099231AF00060002311F086
:1031600082EC91E021E331E202E614E20E942D2B91
:1031700000EC0E941302A0E00FC00A2F07530E9428
:1031800073010EE30E94B70106EC0A1B0E94730153
:103190000CE30E94B701A3950A2F10E020E030E075
:1031A0000E94AF24480159018C01212F220F220BCC
:1031B000322F0E94A4240E94FA26A801B90184019A
:1031C00095010E946626C8F200ED17E00E947F027A
:1031D000C7C20091CA271091CB271A930A9326E001
:1031E00032E202E614E20E942D2B229600E80E94B1
:1031F00013020091BD2710E01A930A9328E132E2EE
:1032000002E614E20E942D2B229600EC0E9413028B
:10321000A7C20E94C30FC8014AE050E08C010E947F
:10322000DB235A934A934AE050E08C010E94DB234F
:103230001A930A932AE232E202E614E20E942D2B4C
:10324000249600E80E9413020091BC2710E01A9314
:103250000A932EE332E202E614E20E942D2B22961C
:1032600000EC0E9413027CC20E94980FC8019A933E
:103270008A932FE432E202E614E20E942D2B22967A
:1032800000E80E94130245E0ECE5F7E200811181BD
:10329000228133810E9417243A932A931A930A9326
:1032A00045E0E8E5F7E200811181228133810E9447
:1032B00017243A932A931A930A9322E632E202E6FB
:1032C00014E20E942D2B289606E80E9413024091DA
:1032D0003627509137274F5F5F4F652F660F660B7C
:1032E000762F00E01CE62CED32E00E94422444E000
:1032F0000E9417243A932A931A930A9320E732E202
:1033000002E614E20E942D2B249600EC0E94130288
:1033100000E61AEE0E947F0223C20091CA27109194
:10332000CB271A930A9320E832E202E614E20E94C5
:103330002D2B229600E80E9413020091AB271091DA
:10334000AC271A930A932BE832E202E614E20E94B9
:103350002D2B229609E80E9413020FED10E01A931C
:103360000A930091A9271091AA271A930A930AEAAF
:1033700010E01A930A9324E932E202E614E20E9472
:103380002D2B269600EC0E9413020091AE270023FD
:1033900021F409E80E94730103C009EC0E94730143
:1033A0000EE30E94B70100E315E70E947F02D8C137
:1033B00040E250E060E070E0E4E5F7E20081118176
:1033C000228133810E9442240E94390F28EA32E28E
:1033D00002E614E20E942D2B00EC0E9413020FED76
:1033E00010E01A930A930091A5271091A6271A932B
:1033F0000A930AEA10E01A930A9323EB32E202E6F8
:1034000014E20E942D2B26960AEC0E94130200E182
:1034100017E20E947F02A4C10FEF0093B62743E09A
:1034200050E060E070E0E0E6F7E200811181228187
:1034300033810E9442240E94390F2DEB32E202E6D2
:1034400014E20E942D2B00EC0E9413020FED10E0FD
:103450001A930A930091A7271091A8271A930A9309
:103460000AEA10E01A930A9323EB32E202E614E22E
:103470000E942D2B26960AEC0E94130200ED17E005
:103480000E947F026DC10091C12710E01A930A9338
:1034900029EC32E202E614E20E942D2B229600E88B
:1034A0000E94130221ED32E202E614E20E942D2B6B
:1034B00006E80E9413022CED32E202E614E20E94BA
:1034C0002D2B00EC0E941302A0E010C00A2F0A531B
:1034D0000E9473010A2F0E94B701A83031F40EEC4C
:1034E0000E9473010FEF0E94B701A3950091C127BD
:1034F0000A1760F703E00E94720232C10091C427EC
:10350000033019F48AE090E00CC00091C427043025
:1035100019F48EE090E005C08091C42790E0880FF8
:10352000991F9A938A932DEE32E202E614E20E94EA
:103530002D2B229600E80E94130221ED32E202E6D2
:1035400014E20E942D2B06E80E94130225EF32E2BE
:1035500002E614E20E942D2B00EC0E941302A0E070
:1035600010C00A2F0A530E9473010A2F0E94B7014C
:10357000A83031F40EEC0E9473010FEF0E94B701E6
:10358000A3950091C4270A1760F703E00E94720216
:10359000E7C00091C22710E01A930A9326E033E2B5
:1035A00002E614E20E942D2B229600E80E941302EC
:1035B00028E133E202E614E20E942D2B00EC0E9487
:1035C0001302A0E010C00A2F0A530E9473010A2FB1
:1035D0000E94B701A83031F40EEC0E9473010FEF86
:1035E0000E94B701A3950091C2270A1760F703E074
:1035F0000E947202B5C00E94980F1A930A932AE2A1
:1036000033E202E614E20E942D2B229600E80E948B
:10361000130221ED32E202E614E20E942D2B06E8AD
:103620000E94130220E333E202E614E20E942D2BF3
:1036300000EC0E941302A0E010C00A2F0A530E945F
:1036400073010A2F0E94B701A83031F40EEC0E94DA
:1036500073010FEF0E94B701A3950091C7270A17C6
:1036600060F703E00E9472027BC00091CA271091AC
:10367000CB271A930A9320E032E202E614E20E947A
:103680002D2B229600E80E94130221ED32E202E681
:1036900014E20E942D2B06E80E94130221E433E27B
:1036A00002E614E20E942D2B00EC0E941302A0E01F
:1036B00010C00A2F0A530E9473010A2F0E94B701FB
:1036C000A83031F40EEC0E9473010FEF0E94B70195
:1036D000A3950091C6270A1760F703E00E947202C3
:1036E00001E00093B1273CC00091B1270023C1F154
:1036F00022E533E202E614E20E942D2B00E80E944C
:103700001302A0E004C000E20E94B701A395A0311B
:1037100090F40A2F00540E9473014A2F0091C82789
:103720001091C9270E94BD230170002361F303E2B9
:103730000E94B701EBCF05EC0E9473010FE20E94DB
:10374000B7010091BE2700540E9473010EE00E9451
:10375000730100E00093B12708EE1DEF0E947F0285
:10376000B0E0E8E0F6E0008103FD5AC000E000931D
:10377000400901E00093AF27E8E0F6E0008103FD97
:103780002DC008EE1DEF0E947F02B3950B2FB02FC6
:10379000003190F30091B42700950093B427009175
:1037A000B427002321F400E00093B32703C007E00F
:1037B0000093B32701E00093B12700E00093B52701
:1037C00000E00093B6270AE510E00E94E50E01E054
:1037D0000093AF2705E00E94720242C10091B42716
:1037E000002349F40091B62700950093B6270AEA12
:1037F0000093B7270DC00CE00E9473010091B3271E
:1038000003950093B3270D3018F001E00093B32720
:1038100008E210E00E94E50E05E00E947202C6C6B2
:10382000E8E2F6E0008100FD16C300E000934009E5
:103830000091B327005081F00A9509F41BC1025092
:1038400009F457C10A9509F499C20A9509F499C176
:10385000075009F4B9C2F7C2E8E2F6E0008100FDC2
:10386000DCC008EE1DEF0E947F02B3950B2FB02F36
:10387000003190F300E310E00E94E50EECE5F7E282
:1038800000811181228133810E94A424A801B90101
:103890004A015B01E8E5F7E2008111812281338171
:1038A0000E94A424A401B5010E942E0F0093382782
:1038B00010933927E8E5F7E20081118122813381F5
:1038C000ECE7F7E20083118322833383ECE5F7E230
:1038D0000081118122813381E8E8F7E200831183BE
:1038E000228333838201212F220F220B322F0E9449
:1038F000A4240E94FA2640913827509139275A93E0
:103900004A9340E050E060E070E40E9464250E9429
:10391000B1241A930A9323E633E202E614E20E94EA
:103920002D2B249600E80E94130200913827109155
:103930003927053C2FEF120764F400E02091382767
:1039400030913927253A1FEF31071CF00060002322
:1039500099F028E733E202E614E20E942D2B00ECF6
:103960000E94130200EB10E00E94E50EE8E2F6E090
:10397000008100FFFBCF74C029E833E202E614E2C5
:103980000E942D2B00EC0E94130200E210E00E9426
:10399000E50E8091A5279091A627009138271091D8
:1039A0003927801B910B8A55904001968093A72759
:1039B0009093A8271091A827112342F4E7EAF7E291
:1039C0000081118108591E4F008311830E94F10F5D
:1039D000E8E2F6E0008100FFFBCF01E00093AF27B3
:1039E00024E731E202E614E20E942D2B00EC0E9453
:1039F00013023091A827232F08E110E00E94060847
:103A00002091A72709E110E00E94060805E00E9426
:103A1000720201E00093AF2723C001E00093AF27BB
:103A20000091CA271091CB271A930A932AE933E20F
:103A300002E614E20E942D2B229600E80E94130257
:103A400000E310E00E94E50E0091B827002311F476
:103A500001E001C000E00093B7270CE00E94720271
:103A60002CEA33E202E614E20E942D2B00E80E94C9
:103A700013029CC50E94210F00E010E00E94330D4C
:103A800008E8602E03E1702E80E090E01AC08C01FF
:103A9000005A164F0093CC271093CD2708EE1DEF48
:103AA0000E947F020091CA271091CB2706151705A7
:103AB0003CF46090CA277090CB27082F0093BD2755
:103AC00003968B3F00E0900714F32091BD2709E097
:103AD00010E00E94060810E600E40E94FA0E4091F1
:103AE000C72750E00FEF10E00E94AF230E94330D74
:103AF0005DC5882499240E94210F84E591E012C0BD
:103B0000809326099093270905E00E9472020E9483
:103B1000980F801691062CF44801809336279093D5
:103B200037270496833F01E0900754F3009136272E
:103B300010913727009326091093270910E400E518
:103B40000E94FA0E30913727232F00E110E00E94E7
:103B500006082091362701E110E00E94060826C5DC
:103B600024ED33E202E614E20E942D2B00E80E94CD
:103B7000130200E810E00E94E50E00E810E00E9449
:103B8000E50EE8E2F6E0008100FDE2C000E61AEE94
:103B90000E947F02B3950B2FB02F053190F301E007
:103BA0000093B22722EB33E202E614E20E942D2BAF
:103BB00000E80E94130200E310E00E94E50E01E01D
:103BC0000093AF2708E20E94720223EC33E202E680
:103BD00014E20E942D2B00E80E94130200E310E083
:103BE0000E94E50E0EE10E94720280E090E0A0E0EB
:103BF0001EC0ECE5F7E200811181228133810E9431
:103C0000A424A801B9014A015B01E8E5F7E20081BB
:103C10001181228133810E94A424A401B5010E9454
:103C20002E0F800F911F0BE00E947202A395AA3005
:103C300000F34AE050E08C010E94DB23C801E091D0
:103C4000A527F091A627EA55F040E81BF90BE09371
:103C5000A527F093A6270091A5271091A62709363E
:103C600021E0120744F0E5EAF7E2008111810856ED
:103C70001140008311831091A627112342F4E5EA35
:103C8000F7E20081118108591E4F008311830E94C1
:103C9000D90F0EE00E947202ECE5F7E2008111817B
:103CA000228133810E94A424A801B9014A015B0149
:103CB000E8E5F7E200811181228133810E94A4248A
:103CC000A401B5010E942E0F38010CEA60160FEF17
:103CD00070060CF045CF25EE33E202E614E20E94B6
:103CE0002D2B00E80E94130205E210E00E94E50E71
:103CF00005E00E94720205E210E00E94E50E0091CC
:103D0000A5271091A6270093A7271093A827009115
:103D1000A7271091A8270E947F0C3091A627232F58
:103D200006E110E00E9406082091A52707E110E0B7
:103D30000E9406083091A827232F08E110E00E9476
:103D400006082091A72709E110E00E94060819CF74
:103D50000091B227002389F426EF33E202E614E251
:103D60000E942D2B00E80E94130208EE1DEF0E9416
:103D70007F0200E510E00E94E50E18C4E8E2F6E0DC
:103D8000008100FD14C008EE1DEF0E947F02B39574
:103D90000B2FB02F053190F300E610E00E94E50EE6
:103DA0000E94C90D10E200E30E94FA0E59CE009164
:103DB000AE2700950093AE2702E310E00E94E50EC7
:103DC00005E00E947202F2C381E090E04091BE27BC
:103DD0008C010E94B723C8014091BE270091C827DB
:103DE0001091C9270E94BD230170002379F08095AE
:103DF0009095E8ECF7E200811181082319230083F4
:103E0000118310E500E40E94FA0E0CC0E8ECF7E222
:103E100000811181082B192B0083118310E300E42A
:103E20000E94FA0E01E00093B1272091C8270CE10F
:103E300010E00E9406083091C927232F0DE110E001
:103E40000E940608B3C301E00093AF2708E210E028
:103E50000E94E50EABC3E8E0F6E0008102FDD0C1B0
:103E600000E0009340090091B327E8E0F2E00C94F1
:103E70008F26E8E0F6E0008102FD1FC000E61AEEA2
:103E80000E947F02A3950A2FA02F033190F3009187
:103E9000BB2700950093BB272091BB2705E110E0CD
:103EA0000E94060801E00093B22700E510E00E949E
:103EB000E50E01E00E9472027CC30091B22700234C
:103EC00081F40091B92703950093B9270A3018F0BF
:103ED00000E00093B9272091B92702E110E00E9489
:103EE000060886C10091BD2703950093BD270B3FAF
:103EF00018F000E00093BD272091BD2709E010E0F5
:103F00000E94060800E41CE90E947F0271C1009132
:103F1000BC2703950093BC270D3318F001E00093F4
:103F2000BC272091BC270AE010E00E94060800E4AC
:103F30001CE90E947F025CC180913627909137274F
:103F400001978093362790933727843501E09007B7
:103F500034F404E511E000933627109337270091DD
:103F6000362710913727009326091093270930919F
:103F70003727232F00E110E00E9406082091362702
:103F800001E110E00E94060833C1E8E0F6E000819C
:103F900001FD11C000E010E00093AB271093AC27A7
:103FA0000093A9271093AA2704E610E00E94E50ECB
:103FB00006E00E9472020091AE27002309F580916D
:103FC000AB279091AC2701968093AB279093AC27B9
:103FD000813008E0900734F000E018E00093AB2750
:103FE0001093AC273091AC27232F02E210E00E94FF
:103FF00006082091AB2703E210E00E94060820C0CB
:104000008091A9279091AA2701968093A927909340
:10401000AA27893601E0900734F000E010E0009311
:10402000A9271093AA273091AA27232F00E210E096
:104030000E9406082091A92701E210E00E940608CC
:104040002091AB273091AC270091A9271091AA2786
:104050000E94740D02E00E947202CAC08091A527DE
:104060009091A62701968093A5279093A62788363E
:1040700001E0900734F000E010E00093A5271093D2
:10408000A6270E94D90F0091A5271091A62700937B
:10409000A7271093A8273091A627232F06E110E029
:1040A0000E9406082091A52707E110E00E9406085B
:1040B0009FC08091A7279091A82701968093A7275A
:1040C0009093A827883601E0900734F000E010E0D4
:1040D0000093A7271093A8270091A7271091A8273E
:1040E0000E947F0C3091A827232F08E110E00E9446
:1040F00006082091A72709E110E00E94060878C071
:104100000091C12703950093C127093018F008E0FA
:104110000093C1272091C12705E210E00E94060804
:1041200067C00091C42703950093C427043018F09A
:1041300003E00093C4272091C42704E210E00E940A
:10414000060856C00091C22703950093C227093084
:1041500018F008E00093C2270BE910E0009326084E
:10416000109327082091C2270BE010E00E94060858
:104170000091C22710E000932A0810932B0838C042
:104180000091C72703950093C727093018F008E06E
:104190000093C7274091C72750E00FEF10E00E941F
:1041A000AF230E94330D2091C7270EE110E00E943B
:1041B00006081EC00091C62703950093C627043049
:1041C00018F003E00093C6272091C62707E210E00D
:1041D0000E9406080DC00091BE2703950093BE27DC
:1041E000003118F000E00093BE2701E00093B127F2
:1041F00008E210E00E94E50E01E00093AF27D6C16F
:10420000E8E0F6E0008101FDD1C100E00093400943
:104210000091B327E8E2F2E00C948F26E8E0F6E0A4
:10422000008101FD25C000E61AEE0E947F02A395E1
:104230000A2FA02F033190F30091C3270395009319
:10424000C327043018F001E00093C3272091C3274F
:104250000FE110E00E94060801E00093B22700E59C
:1042600010E00E94E50E00E61AEE0E947F02A1C156
:104270000091B227002381F40091BA27039500939F
:10428000BA270A3018F000E00093BA272091BA2725
:1042900003E110E00E94060882C10091BD270A9543
:1042A0000093BD270E3F18F00AEF0093BD27209121
:1042B000BD2709E010E00E94060800E41CE90E9406
:1042C0007F026DC10091BC270A950093BC27002393
:1042D00019F40CE30093BC272091BC270AE010E0FE
:1042E0000E94060800E41CE90E947F0258C18091E8
:1042F000362790913727019680933627909337275A
:10430000843F01E0900734F003EF11E0009336277B
:1043100010933727009136271091372700932609ED
:104320001093270930913727232F00E110E00E94D6
:1043300006082091362701E110E00E9406082FC1EF
:10434000E8E0F6E0008102FD11C000E010E000931B
:10435000AB271093AC270093A9271093AA2704E654
:1043600010E00E94E50E06E00E9472020091AE2766
:104370000023F9F48091AB279091AC2701978093AB
:10438000AB279093AC27992332F400E010E0009320
:10439000AB271093AC273091AC27232F02E210E01B
:1043A0000E9406082091AB2703E210E00E94060855
:1043B0001EC08091A9279091AA2701978093A927D1
:1043C0009093AA27992332F408E611E00093A927D5
:1043D0001093AA273091AA27232F00E210E00E9411
:1043E00006082091A92701E210E00E94060820910A
:1043F000AB273091AC270091A9271091AA270E94E2
:10440000740D02E00E947202CAC08091A5279091AB
:10441000A62701978093A5279093A627992332F486
:1044200008E611E00093A5271093A6270E94D90F54
:104430000091A5271091A6270093A7271093A827DE
:104440003091A627232F06E110E00E940608209154
:10445000A52707E110E00E940608A1C08091A727C8
:104460009091A82701978093A7279093A827992335
:1044700032F408E611E00093A7271093A8270091D3
:10448000A7271091A8270E947F0C3091A827232FDF
:1044900008E110E00E9406082091A72709E110E03A
:1044A0000E9406087CC00091C1270A950093C1278D
:1044B0000F3F19F400E00093C1272091C12705E2C6
:1044C00010E00E9406086BC00091C4270A95009373
:1044D000C427013018F401E00093C4272091C427B9
:1044E00004E210E00E9406085AC00091C2270A9513
:1044F0000093C2270F3F19F400E00093C2270091F8
:10450000C227002331F400E010E000932608109346
:1045100027082091C2270BE010E00E9406080091B6
:10452000C22710E000932A0810932B0838C000918E
:10453000C7270A950093C7270F3F19F400E000939F
:10454000C7274091C72750E00FEF10E00E94AF232C
:104550000E94330D2091C7270EE110E00E9406084B
:104560001EC00091C6270A950093C627013018F493
:1045700001E00093C6272091C62707E210E00E94C1
:1045800006080DC00091BE270A950093BE270F3F75
:1045900019F40FE00093BE2701E00093B12708E271
:1045A00010E00E94E50E01E00093AF2700E00093C9
:1045B000B2270091BD2710E0005A164F0093CC2778
:1045C0001093CD270091BB27002311F40C94011404
:1045D000009164060F73009364060AE20093A42717
:1045E0000C94091400008895FECF0E94DC26C801B7
:1045F000D9012A013B015CD057D071F482019301AB
:1046000053D051F401E2E9EDF7E2008341830FEF6B
:104610001FEF2FE73FE73DC044D0A201B3010E9446
:104620000325AC01BD0140D061F442D03AD00E94D4
:104630007E260BED1FE029EC10F43FE32AC03FEB90
:1046400028C0A201B3012DD00E94DD250801190167
:104650002FD0820193010E94662623D0A0F41CD0A3
:1046600050F424D0A801B9010BED1FE029E430E497
:104670000E9447250EC01AD04BED5FE069E470EC54
:104680000E94032506C008D010F410D002C00ED03E
:104690003058E8E00C94ED260E947E2680019101BE
:1046A00008958C019D0108950C945C260C94DE29DC
:1046B00040E050E060E070E008953F7741E00C9406
:1046C0007D2A0FE10DBF01E20EBFC0E0D1E20E94E2
:1046D0007D27002311F00E94602A0E94C8100E94CA
:1046E000F2220C94F2220D01DA0140E050E060E089
:1046F00070E00E945C2639F400E010E04D934C938A
:1047000020E030E00CC0B901660F771F7E57572FAD
:10471000550F550B7D935C932F7730783F63D00115
:1047200008950024E8E0EA9532F0001F001C04160A
:10473000D0F3041AF8CF001F402D00950895FF27ED
:10474000442312F4F1604195002312F4F095019591
:104750000E949123F0FD0195F1FD41950895149F6C
:10476000102D059F100D049F002D110D08954A95E1
:104770001AF0000F111FFBCF08954A951AF01595F6
:104780000795FBCF089500241124EFE0001F111FAF
:10479000001C111C0416150610F0041A150AEA95DF
:1047A000AAF7001F111FA0010095109508955195BB
:1047B000419550400895FF27552312F4F160F7DF2B
:1047C000112312F4F09507D00E94C323F0FD03D00B
:1047D000F1FDEDCF08951195019510400895222423
:1047E000349F302D259F300D169F300D079F300DC3
:1047F000249F202D310D159F200D311D069F200D6A
:10480000311D149F102D210D321D059F100D211DEE
:10481000321D049F002D110D221D321D08954A9551
:104820002AF03695279517950795F9CF08954A955B
:104830002AF03595279517950795F9CF0895002407
:1048400011241001E0E2EA9592F0001F111F221FCF
:10485000331F001C111C221C331C041615062606CF
:10486000370688F3041A150A260A370AECCF001F08
:10487000111F221F331FA001B10100951095209533
:1048800030950895FF27772312F4F16015D0332374
:1048900012F4F09509D00E941F24F69508F404D074
:1048A000F69508F409C00895309520951095019566
:1048B0001F4F2F4F3F4F089570956095509541952C
:1048C0005F4F6F4F7F4F0895FF27112477FB660FCF
:1048D000771F089409F4771F679517F8EE270024CF
:1048E00037FB220F331F089409F4331F279507F86D
:1048F000089527FD0EC0EE0F001F111F221F3A95CD
:104900003230B8F7332319F427FD31E002C027FF16
:1049100030E0E03821F400FF08940EF488940F4F43
:104920001F4F2F4F3F4F323038F4332319F427FDF8
:1049300031E002C027FF30E03F3F29F0220F000C9A
:10494000379527950895ACC0032E002012F40E94DD
:104950005424E02F012F122F232F3EE9D1CF002422
:10496000F8CFBCDF432F4F5748F04F3148F007FCDA
:1049700091C03FE72FEF1FEF0FEF089533278CC053
:10498000322F212F102F0E2F4F5141950E940F24AF
:1049900007FE08950C945424F901EE0FFF1F37FB16
:1049A000FF3F31F0EF2BE12BE02B8894B894089572
:1049B000E02BE12B21F008949894B89408959894F2
:1049C000889438940895FB01EE0FFF1F77FBFF3F9B
:1049D00031F0EF2BE52BE42B8894B8940895E42B69
:1049E000E52B69F3E8CFEFDF68F021F43723262FBA
:1049F0008A010895372FFBCFE6DF20F00BF00895F2
:104A00007327EAF751C0C8DFE8F3B3F361F3DBDFE4
:104A1000C8F383F3A1F358DF401751076207730708
:104A200031F4011411F10024E89488942BC078F03B
:104A3000332E372F732D322E262F632D312E152F27
:104A4000532D302E042F432D302C012C132C3717CF
:104A500039F0669557954795F795E0407395F7CFF0
:104A6000E7FBEE0FE0E010246AF0EF0F041F151FC4
:104A7000261F60F4279517950795E79508F4689425
:104A800033953ECFEF0B040B150B260B39CFE0E827
:104A90007E27B9CF302D307822271127002708959F
:104AA0003FE7302920E8F9CF3FEF2FEFF6CF8BDF3C
:104AB000D8F3D1F370783727089585DFA8F3A3F3EF
:104AC000F9CF3078372793CF67DF70F383F3A9F3FB
:104AD0007ADF50F3B3F3A9F3F7DE0124E8943F57EC
:104AE000E040370FEF1F12F0D9F603C03A3E90F2C4
:104AF0006894E0E00A92AA933A93AA2733242224E6
:104B00003327049FF001059FF00D712D731F149F33
:104B1000F00D711D221C069F700D211C331C159F6A
:104B2000700D211C331E249F700D211C331E169FF7
:104B3000200C311CAA1F259F200C311CA31F269F6F
:104B4000300CA11D39915EF43395A69537942794C6
:104B50007795F795E79533953130BCF316C0AA23C6
:104B600022F0332351F4339510C0339571F4A99199
:104B7000099096CFA7FD09C03A95EE0FFF1F771F4A
:104B8000221C331CAA1F3230A8F7E894FE2B09F030
:104B900068942A2F8101E72FA9910990BACE13DFDB
:104BA00010F00BF087CF80CF0EDFE9F3E0F3032E98
:104BB000072670CF032E072673CFEEDEA0F37BF31C
:104BC00099F301DF80F39BF3A9F37EDE012427FD37
:104BD00006C0000F111F221F3150E040F8CF67FDC3
:104BE00006C0440F551F661F7150F040F8CFE8947F
:104BF000371BEF0B3158EF4F2AF0EE23E9F63F3F1A
:104C0000D9F203C03A3EA8F26894E0E0F0E0112443
:104C1000139440175107620738F0315008F4689434
:104C2000000F111F221FEE1F041B150B260BEF0B8D
:104C3000000F111F221FEE1F0A9279E17A95AAF048
:104C4000041715072607EF0730F0041B150B260B7A
:104C5000EF0B089401C08894111C221C331C001C0B
:104C6000000F111F221FEE1FE9CFF0F9E894E22B8D
:104C7000E12BE02B09F0689406943794279417945D
:104C8000E79508F468947395B9F30990332311F00C
:104C9000F0FF09C0369427941794E79508F46894B8
:104CA00033953130BCF3012D122D232D32CE8BCE16
:104CB00098940895189408956FDED0F3C1F383DEBD
:104CC000B8F3041715072607370708957CDEA0F010
:104CD00063DE90F029F0E32FE7273AF47317089585
:104CE00072DE51F04EF00894089504171507260758
:104CF000370719F016F4B8F78894089564DEE0F3E6
:104D00004BDED0F3E7DFC0F3089408957591659109
:104D100055914591159011FA259035900895F9DF38
:104D2000041B10E003C0F4DF041B150B20E030E08F
:104D300005C0ECDF041B150B260B370BB8F010FC7D
:104D400017C045910590E00FF11F0417100540E0D2
:104D50002407340758F436F404910024F101E01BD1
:104D6000F0090994E00FF11F25903590F1010994A5
:104D700011F4D6F7F1CF31960EF0319650E060E0A5
:104D800070E045914B3F48F089F34F3F29F04E3F8B
:104D900011F07591659155914591041B150B260BEA
:104DA000370B39F318F3E7CFFA92EA92DA92CA9204
:104DB000BA92AA929A928A927A926A925A924A9253
:104DC000BA93AA939A938A930895FF84EE84DD841C
:104DD000CC84BB84AA84998488847F806E805D8023
:104DE0004C80BB81AA8199818881F0E0EC0FFD1F86
:104DF000EF0108950E94D826229741E050E060E03C
:104E000070E00E94662660F440E00E945C2621F477
:104E100002E26BD03FEF5FC001E267D03FE75BC0CB
:104E2000AE010E947323C801D90143EF54E065E34A
:104E30007FE30E94662668F437FBAA0FBB1FB39579
:104E4000B695A795B7F908811981015010400883DC
:104E5000198340E050E060E87FEB43D0280139013E
:104E600040E050E060E87FE33CD0A801B901820156
:104E700093010E94DD25C801D901A801B9012FD0F5
:104E8000280139010881102F110F110B212F312F0B
:104E90000E94A42448E152E761E37FE320D0480167
:104EA000590142E252E964ED7EE38201930117D099
:104EB0004DED5BE96AE27FE316D0A201B3010FD0AA
:104EC00044E050E060E070E40ED0AC01BD0107D0DA
:104ED000A401B50108D02296ECE00C94E9260C94CC
:104EE00064258C019D010C940325E9EDF7E2008314
:104EF00051830FEF1FEF2FE7089501E008950E94FF
:104F0000D426EF97EF976A972A873B874887598778
:104F100068017B0100E00B830C8302C011D21BD21D
:104F20000AD2053251F00023C9F70B811C81EF969C
:104F3000EF966A96E0E10C94E5260081053221F4B3
:104F400002D2FED105E2EBCF00E00F830E830A838D
:104F500009833E0102E1600E00E0701E0AE014E2E7
:104F6000088B198B06C00981002311F40081098385
:104F7000EAD1D9D10052B9F3035059F00850B1F336
:104F8000025019F0035049F00CC00A8103950A83BE
:104F9000EFCF0E8103950E83EBCF0F8103950F8327
:104FA000E7CF00810A3279F4AAD1AD90BD9098D1B3
:104FB000BB203AF4B194A19400E0B00A0A810395B1
:104FC0000A83C1D114C0AA24BB244AE050E00DC01A
:104FD00021916F0185010E94AF23A22EBB24A00E58
:104FE000B11E00EDA00E0FEFB01EA0D188F30A8114
:104FF000002311F000E00F8396D10E32F1F4A3D11B
:1050000092D10A3231F47BD18D909D9069D19BD1A0
:1050100017C0882499244AE050E088D188F421916F
:105020006F0184010E94AF23822E9924800E911E6D
:1050300000ED800E0FEF901EF0CF88248A94982CFC
:1050400080E071D10C5421F00C5131F0045039F44E
:1050500081E0C80E7AD103C001E0C00ED81E6BD12A
:10506000E8E4F2E00C948F2680FB5EF44B815C81D7
:10507000652F660F660B47D140835183628363833C
:105080004FCF2B813C813FD12083318349CF37D112
:105090000D91119625D10A8B2E0103E115D1E0C0A7
:1050A0002ED16D907D901CD1062D072921F40BE1A6
:1050B000602E04E2702E992022F400E1802E07E297
:1050C000902E80E090E001C00196F30101913F0134
:1050D000002319F088159905BCF30CD12301919593
:1050E00081959040680E791EBBC00E81002331F07F
:1050F000082D092919F49924882483940AE214E2DA
:10510000088B198B0881003739F4F9D0ECD000E115
:10511000D5D000E0098330C0F1D046F40D911D9147
:105120002D913D91DDD0C801D90101C0DCD00881AD
:105130000F3611F408E0ECCF053749F70AE0E8CF65
:10514000DDD04D915D9126F46D917D91C9D005C062
:10515000C7D0652F660F660B762FCA01DB01772358
:105160004AF40DE209839095A095B09581959F4FE3
:10517000AF4FBF4F0AE0A2D03E0107E9600E00E04A
:10518000701E2E0107E9A0D0082F092B0A2B0B2B2C
:1051900011F001E001C000E00D83082D092919F488
:1051A0000D8100FF1FC094D0E889F989E00DF11D41
:1051B0000081F30102933F018BD0C801D901012B7B
:1051C000022B032B81F799206AF40F81002351F001
:1051D000A3D010E04501801A910A04C000E3F30156
:1051E00002933F018E0109561F4F06191709081532
:1051F0001905A4F30E81002399F10D8100FF30C041
:105200000881083711F0083549F474D0F30108819A
:10521000008370D000E3F301008322C00F3601F554
:10522000F30100810033E1F000E302933F0118C075
:105230000BE3602E04E2702E462C502EF20100810A
:10524000002371F001E040D0F9CF0FEFC00ED01E67
:105250000EE5602E04E2702E01E6402E04E2502E90
:10526000420186189708A814B9041CF480E090E065
:1052700007C052D0A818B90810E0A01AB10AC50199
:105280000A81002321F401C063D00197EAF7098164
:10529000002339F055D004C053D0F30101913F01F0
:1052A0005AD00FEF800E901EBAF70A81002309F43E
:1052B00037CE01970AF434CE4BD0FBCF10E00C87E9
:1052C0001D871E871F870895400E00E0501E089519
:1052D0004C855D856E857F858C019D010C941F2416
:1052E000A083B18308958D919D91A083B183A0E0A7
:1052F000B0E008950FEF600E701E089580FBF70177
:10530000A081B1810895F701A081B1810D911D9116
:10531000A083B183F80108950981002311F001E011
:10532000089500E00895F60100810895F6010081D6
:1053300000530A300895F60101916F010883089522
:1053400028853985089501E0C00E00E0D01E08953B
:105350002885398500E2EA85FB8509950B811C814A
:105360000F5F1F4F0B831C8308950E94E026C80126
:10537000D9011A013F7740E856E968E17BE40E94D1
:105380007E2638F416D0B38300E010E020E030E051
:105390000DC03B2F0E94B1240E94A4240AD0338365
:1053A000A801B9018C019D010E944725E4E00C94FD
:1053B000F126F10100831183228308950E94D426EF
:1053C000C801D901BF7741E050E060E87FE33B2F9F
:1053D0000E94662670F440E00E945C2629F40BEDE2
:1053E0001FE029E43FE350C0CC24DD24EE24FF2459
:1053F0001CC00BEDC02E0FE0D02E09E4E02EF72EDE
:1054000040E07FEB082F48D02801390140E050E010
:1054100060E87FE38C019D013FD0A801B9018201C2
:1054200093010E94DD25C801D901AC01BD018C01A9
:105430009D012DD02801390144E25FEF6BE27CEB46
:1054400026D048E854E466EA7EE328D048E150ECF0
:105450006FE370E423D045EB1CD0480159014AEEBC
:1054600054EB66E870E48201930118D046EB11D04A
:10547000A801B901840195010E94DD25AC01BD019F
:1054800006D0A601B70108D0E0E10C94E5260C9403
:1054900064255DEF68E670E40C940325FDDFA2014E
:1054A000B301F5CF20E006D0E9F70895259102D0A9
:1054B000E9F708952D9301501040202F212B0895D6
:1054C0008AE797E5FC0105911491FC013296A591BC
:1054D000B491FC01349625913491422F432B19F05D
:1054E000F901E4DF01C0DEDF069617E58638910793
:1054F00048F3089540E00C947D2A0E94DC2628970A
:10550000802FB32F442E40E050E060E070E00E9416
:10551000662610F401E001C000E0000F400EBF77E6
:1055200043E859EF62E27FE3082F3B2F80D076D02B
:1055300041E05CEF6FE777E40E947E2688F5AE01DC
:105540000E94B5296BD0042D10E06BD048815981A1
:105550006A817B8172D0088319832A833B83AE01E1
:105560004C5F5F4F2A0140E050E060E87EE35FD08F
:10557000A2010E94B52940E050E060E870E40C818F
:105580001D812E813F8153D0A801B9010881198165
:105590002A813B810E9447250E94B124402E0CC0E5
:1055A0000E94B124602E3DD0A801B9018C019D015B
:1055B00033D0460C03E0402240FA3EF4AC01BD017A
:1055C00000E010E020E83FE327D002E0401608F0BA
:1055D000B0588C019D0129D0280139014BEF57EDBE
:1055E0006EE179E324D045E656E269E97BEB21D010
:1055F00048E554E363EA7DE31CD041EE5DE565E2F6
:105600007FEB17D04BED5FE069EC7FE316D00DD058
:105610002896E8E00C94ED260E944725C801D901A0
:10562000089520E030E00C94AF24AC01BD010C944F
:10563000642503D0A201B301FACF0C9403251B2FDC
:105640006A2FF901A081B181AD014F5F5F4F4083A7
:1056500051830C93A62FB12F0895BA93AA93249740
:105660000A831B8389019E012A5F3F4F2883398368
:10567000BE01AE014E5F5F4F2FE13BE20E947F27EC
:1056800020E0AA81BB812C932496A991B991089519
:105690000E94D82622974801590141E050E060E07D
:1056A00070E00E94662698F440E00E945C2629F48F
:1056B00000E010E020E030E04EC001E2E9EDF7E26A
:1056C000008351830FEF1FEF2FE73FE744C0AE0188
:1056D0000E947323C801D90145EC53E062E47FE3E3
:1056E0000E9403254AE151E562E17FE33BD0A80136
:1056F000B9018C019D013BD0402E088100FF14C0F0
:105700000A952DD0802F43EF54E065EB7FE3042D05
:105710000E94642537FB220F331F380F36952795DB
:1057200037F9C801D9010BC01AD0842D912FD901A6
:1057300037FBAA0FBB1FB00FB695A795B7F940E08E
:1057400050E060E87EE38C019D010CD0AC01BD010E
:10575000840195010CD02296ECE00C94E92642E0FD
:105760000C949F230E9464252801390108950E940A
:10577000DD25A201B3010C940325420320218657A5
:10578000790362240000202D20504C4153452057BE
:10579000414954202D2000202020202020203C3E64
:1057A000202020202020200045726173696E672030
:1057B000454550524F4D2100726164696F646F6DB1
:1057C0002E75636F7A2E727500204B504F54322D18
:1057D000584D2D762E30392E730020202020202089
:1057E0002020202020202020202000202050726F08
:1057F00066696C65203D20256420202000545820D7
:105800002564487A202025646D41202000525820CC
:1058100025646D5620202020004761696E3D256477
:1058200020005458202D204572726F7221212120B2
:105830002020005258202D204572726F72212121A4
:10584000202020002B253032645B00253032645B41
:105850000023005D532564256446256425630025E7
:10586000642C2564560025646D5620005572783DE1
:1058700025646D5620202E2E2E2E2E2E20002A5AE4
:1058800065726F5F416463203C25643E20202000E8
:10589000556261743D25642E256456202E2E2E2ED1
:1058A0002E2E2000506F7765725F42617420203C7D
:1058B00025643E200025646D4120202020202020EA
:1058C000202020202020200028256C642C256C64BA
:1058D000292E2E2E20002A467265715F54582025ED
:1058E0006C64487A200025646D56202020202020FA
:1058F0000020413D2564202020002A436F696C2050
:10590000626C2E2025633D256425632020002A46F5
:1059100065727269746520200025633D25642563E6
:1059200020200047726F756E6420626C2E20002B61
:10593000256420202020002D2E2E2E2E2E2E2E2EC1
:105940002B00566F6C756D652020202020202020B4
:105950002020002564746F6E6520004265657073B9
:105960002020202020202020202020002B25642003
:105970002020202D2E2E2E2E2E2E2E2E2B00436F4D
:105980006E74722E20202020202020202020200035
:1059900025646D412000506F7765722E20202020F5
:1059A000202020202020004761696E202020202018
:1059B000202020202020200038363432302F303173
:1059C000323334353637383900202020282530321C
:1059D00064293C253032643E20202020200047727C
:1059E0006F756E6420626C2E2D4572726F72004767
:1059F000726F756E6420626C2E202D4F4B2D20002F
:105A00002020202A2A2A202564202A2A2A20202011
:105A100020002B30305B200020204E6F2046657226
:105A20007269746521202020002054616B65204636
:105A30006572726974652120200020202020204595
:105A400072726F7221202020202000202020202030
:105A5000204F4B212020202020202000202020200B
:105A600020206C6F6E6720202020202020002C0139
:105A70003031323334353637383941424344454684
:105A800000286E756C6C20706F696E7465722900E9
:105A900030313233343536373839616263646566A4
:105AA00000464C4F4154533F2077726F6E6720661B
:105AB0006F726D617474657220696E7374616C6C61
:085AC000656421003F3F3F0037
:0400000300000000F9
:00000001FF
